:020000040000FA
:06000000006AD7EF00F0DA
:08000800066A056E158E270E35
:10001000046E100E0CD8030E046EE80E08D8046AA5
:10002000640E05D8046A0A0E02D805500BD0036E80
:100030000650026E0550016E9DEC00F00166159EA3
:1000400015BE1200300F086E8294809880989494A8
:1000500092989298F00E9216085000B222D03A0E62
:10006000026E980E8FEC00F0330E076E30D8130E30
:10007000026E880E8FEC00F02AD8640E8EEC00F031
:1000800026D8640E8EEC00F0220E076E20D8280EC3
:1000900007D80C0E05D8060E03D80082085001D0F0
:1000A0000080076E00A00BD0809803080EE30DD8E7
:1000B000070E026ED00E8FEC00F0D8801200008088
:1000C000FE08D8B4D4EF00F08088073A00A0009072
:1000D0008284F00E801607500F0B8012000000D0B3
:1000E000000000D08294073A000000D0000000D049
:1000F00000B0EDD7320E8EEC00F0D880D4EF00F0D7
:10010000046A036EFF0E0326D8A00426D8A0D4EFFD
:1001100000F0030E026EE70E02D8F4D7026AFD0F5C
:10012000016EFF0E00D001D00126040000D000D0E7
:10013000D8A00226D8A01200F7D7066A056A100ECA
:10014000076E0234053606360350055E0450065A23
:1001500005E20350052604500622D89001360236E7
:10016000072EEFD70150D4EF00F003500702F4CF71
:1001700006F0F3CF05F004500802F4CF02F0F3CFFD
:1001800001F003500802F3500626F4500122E86AF9
:10019000022204500702F3500626F4500122E86AB6
:1001A00002220550D4EF00F0000104001200B0EF6D
:1001B00004F0120C010C100C010C000C000C000CD3
:1001C000400C830C170CD90C070C000C000C010C14
:1001D000020C000C010CDA01DA01090C020C290CEA
:1001E000000C010C010C000CA00C320C090C040CCE
:1001F000000C000C020C030C000C000C000C090C91
:10020000210C000C010C000C010C220C280C000C21
:10021000070C050C810C030C400C000C0A0C070C9D
:10022000050C010C030C400C000C0A0C060C000C15
:10023000FF0C090C000CA10C010C090C010C150C95
:10024000800C250C7F0C350C000C450CFF0C750C3C
:10025000080C950C100C810C020C090C020C150CEE
:10026000800C250C7F0C350C000C450CFF0C750C1C
:10027000080C950C100C910C020CC00C84028C0222
:10028000B802E802040C030C090C040C160C030C55
:10029000540C000C720C000C610C000C6E0C000C69
:1002A000730C000C6D0C000C690C000C730C000C32
:1002B0006F0C000C720C000C180C030C460C000C9C
:1002C0006D0C000C4D0C000C6F0C000C640C000C41
:1002D000750C000C6C0C000C610C000C740C000C08
:1002E0006F0C000C720C000C020C030C04011E516C
:1002F000600B00083EE1050E1F6303D0040E1A6F69
:1003000036D0060E1F6301D035D0080E1F6309D00A
:100310001B0E126F040E136F010E186F196B1D93D5
:1003200026D0090E1F6301D06AD0000E1F6301D0D2
:100330007ED0010E1F6301D09FD0030E1F6301D03A
:100340009BD00A0E1F630BD01C0E126F040E136F8E
:1003500022511227010E186F196B1D9308D00B0E36
:100360001F63120024EE1CF0225120C4DBFF010E9B
:10037000176F1200800E1E631200010E21630FD052
:10038000B20E126F010E136F12C4F6FF13C4F7FF03
:10039000F86A0800F5CF18F4196B1D83E8D7020E30
:1003A000216312D0DA0E126F010E136FDE0EF66E9D
:1003B000010EF76EF86A0900F5CF18F4090009007C
:1003C000F5CF19F41D83D3D7030E21631200F86A09
:1003D000F76A20457C0FF66E020EF7220900F5CF72
:1003E00012F40800F5CF13F412C4F6FF13C4F7FF9C
:1003F000F86A0800F5CF18F4196B1D83B8D7010E01
:10040000176F2FEE71F00F0EDE6AE82EFDD724EE87
:100410001CF0010EDE6AE82EFDD720511B6F03E1B0
:10042000050E1A6F1200060E1A6F08DA12005E6BC4
:100430005F6B1E511F0B000803E11DB15E830ED0E0
:100440001E511F0B010801E109D01E511F0B0208AC
:1004500007E134D8DF50040B01E05E81010E176F15
:10046000010E176312005E0E126F040E136F020E60
:10047000186F196B1D931200010E206309D01E51D5
:100480001F0B000805E11D81030E1F631D916FD72F
:10049000000E206312001E511F0B0208FBE12251C7
:1004A0000F0BF8E00BD8030E1F6303D0840EDF6E32
:1004B0005ED7000E22AF880EDF6E59D724EE00F013
:1004C00022452235E846E846D9261200000E6C6225
:1004D00005D000513C0B340805E010D0040E6C62CE
:1004E000120015D0000E166F000E176F186B196BE7
:1004F000FDDE000E176379D045D977D0020E166362
:10050000AFD057D8C80E00BD880E006F1200040E81
:100510001A6306D020516E6E050ED8B4030E1A6F02
:10052000010E16639DD005D8C80E04BD880E046F59
:1005300012001851106F1951116F000804E307E100
:100540001851400804E2400E106F000E116F105158
:10055000056F185F1151195B0451FC0B1111046FE9
:1005600024EE5EF0115102E1105122E01DA312D0E1
:1005700012C4F6FF13C4F7FFF86A0900F5CFDEFFD7
:1005800009001007FAE11107F8E2F6CF12F4F7CFED
:1005900013F4120012C4E1FF13C4E2FFE6CFDEFF42
:1005A0001007FCE11107FAE2E1CF12F4E2CF13F4F5
:1005B00012000151106F18270051030B116F1923FE
:1005C00014EE5EF014C4D9FF15C4DAFF115102E134
:1005D00010510AE0E6CFDEFF1007FCE11107FAE256
:1005E000D9CF14F4DACF15F41200000E17630AD035
:1005F000400E016F1E0E026F040E036F840E006F1B
:10060000046F2CD01EAF1DD01951255D04E307E106
:100610001851245D04E224C418F425C419F489DFB8
:10062000010E166F400E016F1E0E026F040E036F57
:10063000800E006F5E0E066F040E076FC80E046F0B
:100640000DD0020E166F056BC80E046F400E016FC1
:100650005E0E026F040E036FC80E006F6D981200DD
:10066000000E166F400E016F1E0E026F040E036F18
:10067000880E006F000E046F12000401140E6F6EDE
:10068000000E1A6F1D6B1B6BD9D8120004016DA6EA
:100690000CD8010E1A6312006DBA1200686A696AFA
:1006A00069806988020E1A6F12006D6A696A6D8628
:1006B000010E1A6F120004016D6A696A000E1A6F4A
:1006C00012000401000E1A5D23E068A402D069B490
:1006D00024D86DB2120068A002D069B039D868A8D9
:1006E00002D069B816D868AC02D069BC28D868AA0C
:1006F00002D069BA26D868A202D069B227D8030E00
:100700001A5D06E368A604D069A602D0DFDE68960B
:100710001200698468986D8212006D9269946894E1
:10072000120004011DA11200F8DF6D84100EDA6EB4
:10073000D96AD92EFED7DA2EFCD76D941200689CA8
:10074000120070B08DDF7090689A120068921200EB
:100750006A6A686A9F0E6B6E7B0E696E6E6A2FEE18
:1007600071F00F0EDE6AE82EFDD7160E706E68B6B9
:10077000689668B6FDD76D9873DF1D911B6B030EED
:100780001A6F120004011E511F0B010802E1000E36
:1007900022631200060E1F6327D0210E21630FD0A3
:1007A000FE0E126F010E136F12C4F6FF13C4F7FF93
:1007B000F86A0800F5CF18F4196B1D833CD0220E9F
:1007C000216312D02C0E126F020E136F0C0EF66EF8
:1007D000020EF76EF86A0900F5CF18F40900080058
:1007E000F5CF19F41D8327D01E51600B2008D1E1ED
:1007F000020E1F6309D09E0E126F040E136F010EBE
:10080000186F196B1D9317D00A0E1F6303D021C4F4
:100810009EF411D0030E1F6309D09F0E126F040EB9
:10082000136F010E186F196B1D9305D00B0E1F630C
:10083000120020C49FF4020E176F1200010EE96E21
:1008400014EEA0F0400E1CD8010EE96E14EEE1F09B
:10085000400E00D0E66E2FEE70F0E950D9261A0E49
:10086000DF12E944E846E84604EE04F0E926020E09
:10087000E1CFEBFF030EE2CFEBFF400EEF6E120075
:10088000E66E2FEE70F0E950D9261C0EDF12E94417
:10089000E846E84604EE00F0E926020EE1CFEBFF61
:1008A000030EE2CFEBFFE550E92AE7CFEDFF880E1C
:1008B000EF6E1200016E0401060E1A5D000ED89054
:1008C00009E1E944E846E84604EE04F0E926000EB2
:1008D000D890EFBE1200020EEBCFD9FF030EEBCF84
:1008E000DAFFFF0EDB500160016EE92A0150ED6E68
:1008F00004E0E6CFDEFFE82EFCD7400EEF16EF7CDB
:10090000880EEF120150D8801200016E0401060E0D
:100910001A5D000ED89009E1E944E846E84604EE85
:1009200000F0E926000ED890EFBE1200020EEBCFC9
:10093000D9FF030EEBCFDAFFEC500160016EFF0E22
:10094000DB50ED6E015004E0DECFE6FFE82EFCD771
:10095000400EEF16EF7C880EEF120150D880120087
:10096000926A936A9480948294940A0E1E6E1EC0BA
:1009700081FF806A826A070EC16E070EB46E7DDE4B
:10098000D4EC00F0FE0E23EC00F0010E23EC00F09E
:100990004D0E23EC00F06F0E23EC00F0640E23EC00
:1009A00000F0750E23EC00F06C0E23EC00F0610EED
:1009B00023EC00F0640E23EC00F06F0E23EC00F04B
:1009C000720E23EC00F0200E23EC00F0460E23EC18
:1009D00000F06D0E23EC00F059DE73DED4EC00F075
:1009E00097EC05F07EEC05F0040082B006EF05F010
:1009F000C80E80EC00F01E2A0400FE0E1E5CD8A07B
:100A000004EF05F0FD0E1E6E1EC081FF040082B2D1
:100A100018EF05F0C80E80EC00F01E0604001E5012
:100A20000908D8A416EF05F00A0E1E6E1EC081FF3D
:100A30001EC001F0026A210E036E046A9DEC00F0F4
:100A40001C6E02C01DF01CC007F01DC008F0210E76
:100A5000036E046AB5EC00F0136E06C014F0135078
:100A60001E5C1F6E1FC007F0086A0A0E036E046A40
:100A7000B5EC00F01F6E1FC001F0026A210E036E7C
:100A8000046A9DEC00F01F6E01DE1BDED4EC00F06A
:100A9000FE0E23EC00F0C00E23EC00F0460E23EC1B
:100AA00000F03D0E23EC00F01DC006F01C5005ECDC
:100AB00000F02E0E23EC00F01F5004EC00F0200E8E
:100AC00023EC00F04D0E23EC00F0680E23EC00F058
:100AD0007A0E23EC00F0200E23EC00F0200E23EC25
:100AE00000F0200E23EC00F0200E23EC00F046EC8A
:100AF00003F061EC03F0D4EC00F06ED7100E206E22
:100B000046EC03F061EC03F0D4EC00F0010EE96E6A
:100B100010EE21F02050F9DED4EC00F0206ED8A0C9
:100B200096EF05F021C01EF01EC081FF12001EC00E
:100B300021F0100E206E46EC03F061EC03F0D4ECD3
:100B400000F0010EE96E10EE21F02050B3DED4EC7F
:0A0B500000F0D8A0ACEF05F0120091
:020000040030CA
:08000000E4FEFFF3FFFDBBFF6E
:00000001FF
